:020000040000FA
:02000000AF2B24
:08000800F100030E8301F20078
:100010000000C50F0E28C60F0E2855142130810090
:100020002A08003E03193028241C2E2883160313A7
:10003000DE30850083120313850105145020000073
:10004000000000001E30A100051007305A200514E2
:1000500006305A20A10B242800003C2850203C28C0
:1000600043205E206420722047200F30A1000F3013
:100070005A20A10B372800000B110510720E8300C7
:10008000F10E710E09002D1085192D140800440879
:100090002B02031C4E282B08C40008000000080097
:1000A0002410AA030310A80CA70CA60CA50C031877
:1000B00024140800CC00CC0B5B28080003102B0D87
:1000C000AC006B20B200080003102B0D013EAC0009
:1000D0006B20B300080000308A002C08763E03181D
:1000E0008A0A820032088A00330882000034BE3453
:1000F0000034C7340034CF340034D7340034DF3414
:100100000034E7340034EF340034F7340034FF3483
:100110000134073401340F340134183401341C34F1
:100120000134283401342C340134383401343C3463
:100130000134483401344C340134583401345C34D3
:100140000134683401346C340134783401347C3443
:100150000134883401348C340134983401349C34B3
:100160000134A8340134AC340134B8340134BC3423
:100170000134C8340134CC340134D834B4012D18DE
:10018000C4280730AB00E5290130AB00E5292D1864
:10019000CC280030AB00E5290230AB00E5292D1852
:1001A000D4280030AB00E5290330AB00E5292D1839
:1001B000DC280430AB00E5290330AB00E5292D181D
:1001C000E4280030AB00E5290530AB00E5292D1807
:1001D000EC280B30AB00E5290030AB00E5292D18E9
:1001E000F4280030AB00E5290030AB00E5292D18DC
:1001F000FC280830AB00E5290030AB00E5292D18BC
:1002000004290930AB00E5290030AB00E5292D18A1
:100210000C290A30AB00E5290030AB00E529341485
:100220002D1815290A30AB00E5290030AB00E5296F
:100230002D08B100AB0AE52931082D06031D22293E
:10024000AB01E5292D1830102D1C3014AB0AE5291F
:100250002D08B100AB0AE52931082D06031D32290E
:10026000AB01E5292D182F122D1C2F16AB0AE529FD
:100270002D08B100AB0AE52931082D06031D4229DE
:10028000AB01E5292D18AF112D1CAF15AB0AE529DF
:100290002D08B100AB0AE52931082D06031D5229AE
:1002A000AB01E5292D182F112D1C2F15AB0AE529BF
:1002B0002D08B100AB0AE52931082D06031D62297E
:1002C000AB01E5292D18AF102D1CAF14AB0AE529A1
:1002D0002D08B100AB0AE52931082D06031D72294E
:1002E000AB01E5292D182F102D1C2F14AB0AE52981
:1002F0002D08B100AB0AE52931082D06031D82291E
:10030000AB01E5292D18AE122D1CAE16AB0AE5295E
:100310002D08B100AB0AE52931082D06031D9229ED
:10032000AB01E5292D182E122D1C2E16AB0AE5293E
:100330002D08B100AB0AE52931082D06031DA229BD
:10034000AB01E5292D18AE112D1CAE15AB0AE52920
:100350002D08B100AB0AE52931082D06031DB2298D
:10036000AB01E5292D182E112D1C2E15AB0AE52900
:100370002D08B100AB0AE52931082D06031DC2295D
:10038000AB01E5292D18AE102D1CAE14AB0AE529E2
:100390002D08B100AB0AE52931082D06031DD2292D
:1003A000AB01E5292D182E102D1C2E14AB0AE529C2
:1003B000AB014D1400000000000000000000000030
:1003C000000000000000000000000800BC01BD01AA
:1003D0000830BE000310C00CBD0DBC0DBF0CBD0D20
:1003E000BC0DBE0BEA290800D600D7010830BE00BC
:1003F0000310D60CD70DBE0BF82957080800A6012C
:10040000A701A801A030A500D209521C2614521839
:10041000A614501E2615501AA615D01D2616D01942
:10042000A616501D26175019A617D01C2714D01831
:10043000A714501C27155018A715D11E2716D11A1E
:10044000A716511E2717511AA717D11D2814D11905
:10045000A814511D28155119A815D11C2816D118FA
:10046000A816511C28175118A8172130AA000800F7
:10047000FF30C1000000C10B3A2A0800C70A470834
:10048000123C0319C7014708D3000800C7034708F7
:10049000013E031D4E2A1130C700D30008002E086C
:1004A000C700D300EE3E031C592A1130C70247088B
:1004B000522A08008B13C830850583160313373082
:1004C00085047308850583120313350885048B178B
:1004D0000800FF30F3000030B50008004208BB0000
:1004E0006922B719F310B71B7311B71A731273107F
:1004F00035145A22303038226922371A73103718CF
:100500007311381B73123619F312F310B5145A22F3
:1005100030303822692236187310B81BF310B71820
:100520007312361BF312731135155A2230303822EC
:100530006922371B7310B81AF31037197311361A62
:10054000F312731235165A22303038226922B61B44
:100550007310B618F310B61A7311B6197312F3129A
:10056000B5165A2230303822BB0B702A08004708D3
:10057000013EF421B6000030B700B800FF30541837
:10058000B8007F30C2006E2208004708031DD32A3E
:1005900003010D23CA00D401CA1B54144A08031DC9
:1005A000E82A3E22C52A0330C800DE30C900031005
:1005B000470DF4008B13D7238B17CA000310470D88
:1005C000013EF4008B13D7238B17C9004A08C800DB
:1005D00008004708031DEF2A74080D23F32A740846
:1005E0008B13D7238B17F40A0800831603131C15EB
:1005F0008B1374089B0075089A0055309D00AA3033
:100600009D009C148B1783120313FF30B600B700B4
:10061000B8003F30C2006E220800831603139B000F
:100620009C131C141A0883120313080003010D23E2
:10063000CA00CA1F1E2BCA13D401202BCA17541478
:10064000F4014A08F500F522B722B7220800C522B6
:10065000F401E922CB00E922C300C30A4D1C4C2B54
:1006600007302F02031D372B4F22CD01272BAF0858
:10067000031D4C2B20302E0203193E2221302E0266
:100680000319462200302E020319C7010C302E0236
:1006900003191623CD01272B341C572BB722B72261
:1006A000341C572B3E22B7223418522B272BE92219
:1006B000B600E922B700E922B8004308C2006E2262
:1006C0002A08003E031D702B551C702BD501541CAD
:1006D0006B2B3E22272B0730D0005308D100FF217F
:1006E000381C2E2B272B2B08F421B6004408F421AC
:1006F000B700B8010130C2006E22341C892BC4013E
:10070000AB012A08003E031D892BD0010C30D1001B
:10071000FF214D1C732BCD01FF30B600B700B80090
:100720007F30C2006E220030B600B700B8003F3004
:10073000C2006E22FF30B600B700B8007F30C200A2
:100740006E222E08F421B6002F08F421B700B8015C
:10075000FF30C2006E226E22C401AB01732B8501F3
:100760008101A201AA01B001AF01AE01B101AB014B
:10077000C401B401CD01D50107309900640083168E
:100780000313823081000F168F160F179F01051279
:10079000831203138B168B17C701FF30B600B70007
:1007A000B8007F30C2006E22341C272B732B480800
:1007B0008A007408490703188A0A82000434023444
:1007C000043402340434403404347E340434EC34CD
:1007D0000434F43405343234053452340534993455
:1007E0000534A7340534EB34063423340634673437
:1007F0000634DB340634E6340634F134073432345C
:1008000007346D34013410340034003420340034A3
:100810000034403400340034803400340134003477
:10082000003402340034003404340034003408341A
:1008300000340034103400340034203400340034E8
:100840004034003400348034003401340034003447
:1008500002340034003404340034003408340034EA
:100860000034103400340034203400340034403478
:100870000034003480340034003400340034013457
:100880000134203400340034203400340034603427
:1008900000340034E03400340134E03400340334F4
:1008A000E03400340734E03400340F34E0340034F2
:1008B0001F34E03400343F34E03400347F34E0341B
:1008C0000034FF34E0340134FF34E0340334FF34C7
:1008D000E0340734FF34E0340F34FF34E0341F34A5
:1008E000FF34E0343F34FF34E0347F34FF34E0340D
:1008F000FF34FF34E0340034003401340134103468
:1009000000340034203400340034403400340034E7
:1009100080340034013400340034023400340034B4
:10092000043400340034083400340034103400340B
:100930000034203400340034403400340034803437
:100940000034013400340034023400340034043400
:1009500000340034083400340034103400340034DF
:100960002034003400344034003400348034003407
:100970000034403400340034203400340034103467
:1009800000340034083400340034043400340034BB
:100990000234003400340134003400340034803434
:1009A0000034003440340034003420340034003447
:1009B000103400340034083400340034043400347B
:1009C0000034023400340034013400340034003484
:1009D00080340034003441340134303455345534DB
:1009E0005034AA34AA34A134013400340034003421
:1009F0002034003400344034003400348034003477
:100A0000013400340034023400340034043400343F
:100A100000340834003400341034003400342034FE
:100A20000034003440340034003480340034013465
:100A30000034003402340034003404340034003410
:100A400008340034003410340034003420340034CE
:100A50000034403400340034803400340034003436
:100A600000340134013430348034003420344034D4
:100A700000344034203400348034103401340034E5
:100A800008340234003404340434003402340834AA
:100A900000340134103400340034A0340034003405
:100AA0004034013401341034003400342034003434
:100AB00000344034003400348034003401341034C5
:100AC0000034023420340034043440340034083418
:100AD00080340034113400340034223400340034C3
:100AE0004434003400348834003401341034003489
:100AF0000234203400340434403400340834803468
:100B000000341134003400342234003400344434CE
:100B1000003400348834003400341034003400349D
:100B20002034003400344034003400348034003445
:100B3000013401341034113411341034223422348D
:100B4000203444344434403488348834813401348B
:100B50000734113411341034223422342034443414
:100B6000443440348834883480341134113410349F
:100B70002234223420344434443440348834883499
:100B8000803411341134103422342234203444346B
:100B900044344034883488348034443444344034D9
:100BA00022342234203411341134103488348834FF
:100BB00080344434443440342234223420341134D8
:100BC000113410348834883480344434443440340C
:100BD000223422342134013420342A34AA34A0347B
:100BE0004A34AA34A0345234AA34A0345434AA3437
:100BF000A03455342A34A03455344A34A034553402
:100C00005234A03455345434A0345534553420343F
:100C1000553455344034A53455344034A934553412
:100C20004034AA3455344034AA3495344034AA347C
:100C3000A5344034AA34A9344034AA34AA348034C8
:100C4000AA34AA34A134013420348034003400346E
:100C5000C03400340034E03400340034F034003464
:100C600000347834003400343C34003400341E3412
:100C7000003400340F34003400340734803400343E
:100C80000334C03400340134E03400340034F03430
:100C9000003400347834003400343C340034003400
:100CA0001E34003400340F340034003407348034F0
:100CB00000340334C03400340134E03400340034F0
:100CC0006034003400342034003400340134013402
:100CD00003340034003420340034003460340034F1
:100CE0000034E03400340134E03400340334E034C0
:100CF00000340734E03400340F34E03400341F345F
:100D0000E03400343F34E03400347F34E0340034E5
:100D1000FF34E0340134FF34E0340334FF34E03492
:100D20000734FF34E0340F34FF34E0341F34FF3431
:100D3000E0343F34FF34E0347F34FF34E034FF34B8
:100D4000FF34E034FF34FF34C034FF34FF348034E8
:100D5000FF34FF340034FF34FE340034FF34FC34FD
:100D60000034FF34F8340034FF34F0340034FF34FE
:100D7000E0340034FF34C0340034FF3480340034B5
:100D8000FF3400340034FE3400340034FC340034CA
:100D90000034F83400340034F03400340034E034EB
:100DA00000340034C0340034003480340034003463
:100DB0000034003401340134103492344934203486
:100DC000243492344034493424348134013410348E
:100DD00092344934203449342434803424349234D5
:100DE00041340134053400340034203400340034FC
:100DF00080340034023400340034083400340034C9
:100E000020340034003480340034023400340034A0
:100E1000083400340034203400340034803400348A
:100E200000340034003400340034003440340034E2
:100E300001340034003404340034003410340034FD
:100E400000344034003401340034003404340034BD
:100E500000341034003400344034003400340034A2
:100E600000340134013405340034003420340034BB
:100E70000034803400340234003400340834003448
:100E80000034203400340034803400340234003420
:100E9000003408340034003420340034003480340A
:100EA0000034003440340034003410340034003452
:100EB000043400340034013400340034003440344D
:100EC000003400341034003400340434003400346E
:100ED000013400340034003441340134103400341F
:100EE000003460340034013480340034063400347B
:100EF0000034183400340034603400340134803459
:100F000000340634003400341834003400346034C3
:0A0F100000340034003400340134D2
:02400E00C430BC
:1042000001003200800000000000400000000000BB
:104210002000000000001000000000000800000066
:104220000000040000000000020000000000010087
:1042300000000000000080000000000040000000BE
:104240000000200000000000100000000000080036
:104250000000000004000000000002000000000058
:10426000010000000000000080000000000040008D
:0C42700000000000200000000000010021
:00000001FF
